:0614000002148B024B6692
:01140B0032AE
:0114130032A6
:01141B00329E
:011423003296
:01142B00328E
:031433000243F27F
:01143B00327E
:011443003276
:03144B0002530D3C
:03145300021A93E7
:03145B00021D6D02
:011463003256
:03146B00024475C3
:011473003246
:01147B00323E
:03148300024E9284
:0314E70002148666
:03148600022E0330
:1014EA00AF83E58290F554F0EFA3F075E10490DF45
:1014FA003BE0FFBF01F890F554E0FEA3E0FF90DF68
:10150A0006EEF075E10290DF3BE0FFBF0DF8227EA8
:10151A00007F0090FC28E0FCA3E0FD8E028F03C34D
:10152A00EA9CEB9D503AEE2400FCEF34F0FD90FC6F
:10153A0026E0F513A3E0F5148A828B83C007C00660
:10154A00C005C004125842AA82AB83D004D005D089
:10155A0006D0078C828D83EAF00EBE00B60F80B3E8
:10156A0022E58290F556F0E0FFE59CC39FF59CE5E5
:10157A009C24FAF59C439E10D2BA22AF9E74EF5F68
:10158A00F59E22AF83E58290F55AF0EFA3F090FC26
:10159A0021E06013905A041244E490FC21E0F582A1
:1015AA001245267582EF2290FC217406F090DF3BEB
:1015BA00E0FFBF130280F6C29190F557E0FEA3E068
:1015CA00FF90FC88EEF0EFA3F090FC8274F1F0E457
:1015DA00A3F090FC187472F074F3A3F090FC80E40A
:1015EA00F0A3F090FC33F090FC7CF090FC32F09089
:1015FA00FC7E04F0E4A3F090FC7D7402F090F55CAC
:10160A00E4F090000012173290F55AE0FEA3E0FFD2
:10161A0090F559E0FD7B007C008D017A00C3EB99BF
:10162A00EC9A50548B02EA75F0F0A42EF9E43FFAD2
:10163A0090F55C74F0F089828A83C007C006C00501
:10164A00C004C003121732AA82D003D004D005D036
:10165A0006D007EA601B905A56C0021244E4D00230
:10166A0090FC21E4F08A82C002124526D0028A82C6
:10167A00220BBB00A40C80A190FC8BE0FF30E3336B
:10168A0090FC88E0FEA3E0FFEE540F602690FC88F1
:10169A00E0FEA3E053060F7F007410C39EFEE49F92
:1016AA00FF90FC88E0FCA3E0FD90FC88EE2CF0EFB4
:1016BA003DA3F090FC88E0FEA3E0FFC374FF9EE424
:1016CA009F502390FC88E0FEA3E090DF02EEF090AA
:1016DA00DF04E0FF74FC5FF0E0FF74024FF090FC5F
:1016EA008A7401F0801290FC88E0FEA3E0FF90DF8C
:1016FA0002EEF090FC8AE4F075E1037E607FEA90E6
:10170A00DF3BE0FDBD130280091EBEFF011FEE4F45
:10171A0070EDD291EE4F700C90FC467413F0905A13
:10172A006E1244E475820022AF83E58290F55DF083
:10173A00EFA3F090F55CE0FF240F500A905A7F1255
:10174A0044E47582FF22EF703E90FC32E4F090FC94
:10175A0032E0FE90FC7DE0FDC3EE9D502190FC320C
:10176A00E075F0F1A42472F58274F335F0F583E4A0
:10177A00F090FC32E0FE0E90FC32EEF080D090FC4D
:10178A0032E4F07582002290FC21E0FE601DBE0664
:10179A001E90FC32E0601890DF3BE0FEBE13028030
:1017AA000E90FC217407F07582ED227582ED22906D
:1017BA00FC32E075F0F1A42472FD74F335F0FE8D6D
:1017CA00828E83E0600A90FC467418F07582FE22CD
:1017DA008D828E8374FFF090FC32E075F0F1A424C0
:1017EA0072FD74F335F0FE0DBD00010E7C0090F51C
:1017FA005DE0FAA3E0FB8A138B148C158F037F003C
:10180A008B168F178D828E838CF0C007C0031257F8
:10181A0069D003D00790FC8BE0FE20E3030218DABC
:10182A0090FC32E075F0F1A42472FD74F335F0FEF9
:10183A000DBD00010E90FC5DEBF0EFA3F08D828EE2
:10184A0083125487AE8290F55CEEF090FC8BE0FF39
:10185A00530704BF043F90FC32E075F0F1A42472F0
:10186A00FD74F335F0FF0DBD00010F8E037C00906F
:10187A00FC8BE0FA5302F090FC61EDF0EFA3F090DC
:10188A00FC63EBF0ECA3F090FC65EAF08D828F83A9
:10189A001254C1803B90FC32E075F0F1A42472FD31
:1018AA0074F335F0FF0DBD00010F7C0090FC8BE056
:1018BA00FB5303F090FC68EDF0EFA3F090FC6AEEA6
:1018CA00F0ECA3F090FC6CEBF08D828F8312550A3A
:1018DA0090FC32E075F0F1A42472FE74F335F0FF47
:1018EA0090F55CE0FD8E828F83F090FC32E0FF0F72
:1018FA0090FC32EFF090FC7DE0FEEFB5060590FC1F
:10190A0032E4F075820022AF83E58290F55FF0EF52
:10191A00A3F090FC21E0FF6014BF0102800F905AEF
:10192A00991244E490FC21E0F582124526121585AD
:10193A0090FC2AE4F0A3F090FC2AE0FEA3E0FF8EDC
:10194A00828F83121A1390DF3BE0FFBF0DF890DFFE
:10195A003AE0FF53077FBF6000402790FC2AE0FE71
:10196A00A3E0FF0EBE00010F90FC2AEEF0EFA3F0F9
:10197A00D29190000A12518DC29190000A12518D93
:10198A0080B590FC217402F090FC47E0FCA3E0FDD6
:10199A00A3E0A3E090FC2CECF0EDA3F090F55FE05F
:1019AA00FEA3E0FF90FC30EEF0EFA3F02290FC21C2
:1019BA00E4F090FC47E0FCA3E0FDA3E0A3E090FC88
:1019CA002CECF0EDA3F02290FC217404F090FC477B
:1019DA00E0FCA3E0FDA3E0A3E090FC2CECF0EDA377
:1019EA00F02290FC217405F090FC34E4F0A3F0900E
:1019FA00FC47E0FCA3E0FDA3E0A3E090FC2CECF0A4
:101A0A00EDA3F075820002156BAF83E58290F56154
:101A1A00F0EFA3F090F561E0FEA3E0FFEE2400F5FD
:101A2A0082EF34F0F583E0FF7E008F828E8302140A
:101A3A00EAAF83E58290F563F0EFA3F090F563E0F7
:101A4A00FEA3E0FF90F370EEF0EFA3F0222290FCE9
:101A5A002AE0FEA3E0FF0EBE00010F90FC2AEEF082
:101A6A00EFA3F0C3EE9470EF9403400790FC2AE4CE
:101A7A00F0A3F090FC2AE0FEA3E0FFEE2400F5823A
:101A8A00EF34F0F583E0F58222C021C0E0C0F0C057
:101A9A0082C083C007C006C005C004C003C002C01C
:101AAA0001C000C0D075D00090FC1DE02401F0A355
:101ABA00E03400F090FC22E0FEA3E0FF90FC1DE081
:101ACA00FCA3E0FDECB5060BEDB5070790FC1DE4A1
:101ADA00F0A3F090FC1DE0FEA3E0FFBE0005BF00EE
:101AEA0002800BBE0105BF00028068021C5590FCF3
:101AFA001DE0FEA3E08E077E00AC9C7D00EC420652
:101B0A00ED420790FC2EEEF0EFA3F090FC2AE0FEE7
:101B1A00A3E0FF0EBE00010F90FC2AEEF0EFA3F047
:101B2A0090FC28E0FCA3E0FDC3EE9CEF9D400790EB
:101B3A00FC2AE4F0A3F090DF3BE0FFBF1303021D91
:101B4A005090FC2AE0FEA3E0FF8E828F83121A13C4
:101B5A00021D5090FC21E0FFBF05028003021D50C8
:101B6A0090001912518D90F567741CF090FC2AE0D0
:101B7A00FEA3E090F568EEF090FC2AE0A3E090F571
:101B8A0069F090F56A7442F090F56B744CF090F538
:101B9A006C7441F090F56D7448F090F56E7442F0F3
:101BAA0090F56F744CF090F5707441F090F5717483
:101BBA0048F090F5727442F090F573744CF090F519
:101BCA00747441F090F5757448F090F5767442F0AB
:101BDA0090F577744CF090F5787441F090F579743B
:101BEA0048F090F57A7442F090F57B744CF090F5D9
:101BFA007C7441F090F57D7448F090F57E7442F063
:101C0A0090F57F744CF090F5807441F090F58174F2
:101C1A0048F090F5827420F090FC36741CF0E4A32E
:101C2A00F090FC38F0A3F090FC3AF0A3F090F5683D
:101C3A0012479E90FC34E0FEA3E0FF0EBE00010FA7
:101C4A0090FC34EEF0EFA3F0021D5090FC21E0FF6F
:101C5A00BF03028065BF04028008BF050280030239
:101C6A001D5090FC2CE0FEA3E0FF90FC47E0FAA395
:101C7A00E0FBA3E0FCA3E0FD8E008F01E4FEFFEA97
:101C8A00C398FAEB99FBEC9EFCED9FFDC374649A32
:101C9A00E49BE49CE49D5022905AC71244E490FCD1
:101CAA00217405F090FC47E0FCA3E0FDA3E0FEA34D
:101CBA00E0FF90FC2CECF0EDA3F090FC33E075F023
:101CCA00F1A42472FE74F335F0FF8E828F83E060F4
:101CDA007590001912518D90FC33E075F0F1A4242F
:101CEA0072FE74F335F0FF90DF04E05401FDB40195
:101CFA0000E4332EFDE43FFC8E828F83E090FC36B5
:101D0A00F0E4A3F090FC38F0A3F090FC3AF0A3F0D2
:101D1A008D828C8312479E90FC33E075F0F1A424E7
:101D2A0072F58274F335F0F583E4F090FC33E0FF4A
:101D3A000F90FC33EFF0BF0200400590FC33E4F053
:101D4A00905AE51244E4D0D0D000D001D002D0039A
:101D5A00D004D005D006D007D083D082D0F0D0E00E
:101D6A00D021323290FC21E4F090FC32F090FC3326
:101D7A00F090FC2AF0A3F090FC267453F0E4A3F050
:101D8A0090FC287453F0E4A3F090FC2EF0A3F0909A
:101D9A00FC2CF0A3F090FC227406F0E4A3F090FC73
:101DAA0024F0A3F090FC30F0A3F090FC34F0A3F000
:101DBA0012151990FC21E4F0759DDC859E9E439EC8
:101DCA000443CB1022021D6E9021F612335490FC6C
:101DDA0047E4F0A3F0A3F0A3F0121DCF90F583E43B
:101DEA00F090F5847412F074F8A3F02290FC21E0CC
:101DFA00FFBF000302212BBF0103021FFCBF020326
:101E0A00021EFABF030302212BBF040302212BBFC8
:101E1A00050302210CBF060122BF40028006BF4112
:101E2A000280422275E10490DF3BE0FFBF01F89097
:101E3A00DF0374E5F090DF047404F090DF07741296
:101E4A00F090DF08E4F090DF147410F090DF17E0F0
:101E5A00FF74C04FF090FC217441F090F584741225
:101E6A00F074F8A3F090F583E4F090FC34E0FEA35C
:101E7A00E0FF90F583E0FDFB7C00C3EB9EEC9F50F6
:101E8A004590DF06EDF075E10490DF3BE0FFBF010E
:101E9A00F875E10290DF3BE0FFBF0DF890000212F7
:101EAA00518D90F584E0FEA3E0FF90F583E02EFECD
:101EBA00E43FFF90DF3AE0FD8E828F83F090F58356
:101ECA00E02401F080A475E10490DF3BE0FFBF014C
:101EDA00F890FC34E0FEA3E08E3375340090F5846C
:101EEA00E0F535A3E0F536753201758243022E35E9
:101EFA00E50E7003021FEA90FC45740DF0AF9A7468
:101F0A00FE5FF59AE50E20E403021FEA90FC2174B5
:101F1A0003F090FC1FE0FEA3E08E8212156B905A2C
:101F2A00F31244E490FC1FE0FEA3E0FF8E828F834D
:101F3A0012454190F811E025E0FEE42412FFEE3448
:101F4A00F8FE8F828E831244E490F811E0FFB40108
:101F5A0000E433FF90F583F0EF2416FDE434FCFE31
:101F6A008D828E83E0707290DF04E0FE30E0378F5E
:101F7A0006EE2EFDE42412F582ED34F8F583E0FE38
:101F8A008E337534008F06EE2EFDE42412FEED34F6
:101F9A00F8FD74012EF535E43DF53675320175828A
:101FAA0042122E35802290DF02E0FE8E33E4F534B1
:101FBA00EF2FFEE42412FFEE34F8FE8F358E3675CD
:101FCA003201758242122E3590F583E0FF2416F510
:101FDA0082E434FCF5837401F0AF0E74EF5FF50E02
:101FEA00D20010AF02C200750E00A20092AF439A4F
:101FFA000122E50E70030220FA90FC45740DF0AF41
:10200A009A74FE5FF59AE50E20E4030220FA90F82E
:10201A0011E0FF90F583B40100E433F0905B0812FD
:10202A0044E490F583E025E0FEE42412FFEE34F860
:10203A00FE8F828E8312454190F583E025E0FEE40F
:10204A002412FFEE34F8FE8F828E831244E490F855
:10205A0011E0FFB40100E433FF90F583F0EF24169A
:10206A00FDE434FCFE8D828E83E0707290DF04E022
:10207A00FE30E0378F06EE2EFDE42412F582ED34B1
:10208A00F8F583E0FE8E337534008F06EE2EFDE4FC
:10209A002412FEED34F8FD74012EF535E43DF536D3
:1020AA00753201758242122E35802290DF02E0FEDF
:1020BA008E33E4F534EF2FFEE42412FFEE34F8FEFB
:1020CA008F358E36753201758242122E3590F58320
:1020DA00E0FF2416F582E434FCF5837401F0D200A3
:1020EA0010AF02C200AF0E74EF5FF50EA20092AFFE
:1020FA00D20010AF02C200750E00A20092AF439A3E
:10210A00012290FC34E0FEA3E0FF90FC28E0FCA34F
:10211A00E0FDC3EE9CEF9D50012290FC217404F077
:10212A0022E50E70012290FC45740DF0E50E543044
:10213A0070012290F811E0FFB40100E433FF90F53A
:10214A0083F0EF2416FDE434FCFE8D828E83E0607A
:10215A00030221E390DF04E0FE30E0378F06EE2E23
:10216A00FDE42412F582ED34F8F583E0FE8E337532
:10217A0034008F06EE2EFDE42412FEED34F8FD74D1
:10218A00012EF535E43DF536753201758242122E7F
:10219A0035803590FC77E0E0600A90FC7AE0FDA398
:1021AA00E0FE800890DF02E0FCFD7E00EF2FFCE4F9
:1021BA002412FFEC34F8FC8F358C367532018D33DE
:1021CA008E34758242122E3590F583E0FF2416F57F
:1021DA0082E434FCF5837401F0D20010AF02C2002D
:1021EA00AF0E74CF5FF50EA20092AF2290F7C3E054
:1021FA00FDA3E0FEA3E0FF90F7C8E0FCBC4202802A
:10220A0003022B9190F7C9E0FC24BE5003022B83F2
:10221A00EC240A83F582EC244683F583E4738383F2
:10222A00FC4483AF6A889BD40D3174128383D857D8
:10223A007EF1162995093E83838383838383E8711C
:10224A00B8AED183838383838383838383838383A6
:10225A008383838383838383838383838383ACE6B8
:10226A002B2B22252B2324242424252525262B2BFE
:10227A00282929292A2A2A28292B2B2B2B2B2B2BB5
:10228A002A2B2A29292B2B2B2B2B2B2B2B2B2B2B9A
:10229A002B2B2B2B2B2B2B2B2B2B2B2B2B2B2B2B84
:1022AA002222C007C006C005121585D005D006D067
:1022BA000790FC217440F08D828E838FF01259A111
:1022CA00FC7B0090FC34ECF0EBA3F090F7E9EDF026
:1022DA00EEA3F0758201124236022B9190FC21E4A2
:1022EA00F090F7E9EDF0EEA3F075820112423602A2
:1022FA002B9190FC21E06009905B221244E4022BAE
:10230A00918D828E838FF01259A1FC7B0090F58605
:10231A00ECF0EBA3F08D828E83A3E0FAE4F92CFCB7
:10232A00EA3BFB90F586ECF0EBA3F08D828E83A35B
:10233A00A3A3A3E0FA8A0889098D828E83A3A3A3A3
:10234A00A3A3E0FAE42508F508EA3509F50990FCA3
:10235A001AE4F0A3F074062DF9E43EFA90FC36EC88
:10236A00F0EBA3F090FC38E4F0A3F090FC3AE50817
:10237A00F0E509A3F089828A83C007C006C0051266
:10238A00479EAC82D005D006D0078D828E838FF00F
:10239A00EC12580A90F7E9EDF0EEA3F075820112FB
:1023AA004236022B918D828E838FF01259A190FCB6
:1023BA007AF0E4A3F08D828E83A3E0FB7C0090FC8C
:1023CA007AE0F9A3E0FA90FC7AEC29F0EB3AA3F070
:1023DA0090FC7AE0A3E090FC7AE0F5F0A3E045F007
:1023EA00604B90FC777401F090FC78E0A3E090FCDD
:1023FA0078E0F5F0A3E045F070471246D790FC7AF2
:10240A00E0FBA3E0FC90FC78EBF0ECA3F090FC7806
:10241A00E0FBA3E090DF02EBF090DF04E0FC74FC49
:10242A005CF0E0FC74024CF012468D801490FC774C
:10243A00E4F090FC78F0A3F090FC7AF0A3F0124656
:10244A00D790F7C8E0FC90F7C9E0F53275357A7590
:10245A0036FC7533017534008C82122E35022B91AD
:10246A008D828E838FF01259A190FC8BF090F7E940
:10247A00EDF0EEA3F0758201124236022B9190F72D
:10248A00E9748BF074FCA3F0758201124236022BB8
:10249A009190FC8BE0FC5304F090FC597406F09088
:1024AA00FC5AECF08D828E838FF0C007C006C005FF
:1024BA0012542FD005D006D00790F7E9EDF0EEA31D
:1024CA00F0758210124236022B9190FC8BE0FC537D
:1024DA0004F090FC597404F090FC5AECF08D828E52
:1024EA00838FF0C007C006C00512542FD005D0064E
:1024FA00D00790F7E9EDF0EEA3F07582101242369C
:10250A00022B918D828E838FF01259A190FC8CF050
:10251A00E0FC74015CF090F7E9EDF0EEA3F075824F
:10252A0001124236022B9190F7E9748CF074FCA3E5
:10253A00F0758201124236022B918D828E838FF0C2
:10254A001259A1FC7B008C828B83C007C006C00590
:10255A00121A3BD005D006D00790F7E9EDF0EEA3AA
:10256A00F0758201124236022B9190FC21E0601C28
:10257A008D828E838FF074EF12580A90F7E9EDF08E
:10258A00EEA3F0758201124236022B918D828E8360
:10259A008FF01259A1FC7B0090F586ECF0EBA3F0CA
:1025AA008D828E83A3E0FAE42CFCEA3BFB90F5864D
:1025BA00ECF0EBA3F08D828E83A3A3E0FA90FC1AD1
:1025CA00E4F0A3F074032DF8E43EF990F557ECF02B
:1025DA00EBA3F090F559EAF088828983C007C00618
:1025EA00C00512158DAC82D005D006D0078D828E1B
:1025FA00838FF0EC12580A90F7E9EDF0EEA3F0752C
:10260A008201124236022B918D828E838FF01259EB
:10261A00A1FB7C0090F586EBF0ECA3F0EB4C600399
:10262A0002271A90FC88E0A3E090FC88E0F5F0A36A
:10263A00E045F0601C90DF3BE0FABA1314900028E2
:10264A00C007C006C00512518DD005D006D007803C
:10265A00D290FC88E0A3E090FC88E0F5F0A3E04586
:10266A00F0606B905B47C007C006C0051244E49057
:10267A00FC88E0F9A3E0FA89828A8312454190F343
:10268A0072E0F58212452690F463E0F5821245263F
:10269A00D005D006D00790FC467412F08D828E8346
:1026AA008FF074EC12580AC291C007C006C0051216
:1026BA004668D005D006D00790FC21E4F090F7E9EF
:1026CA00EDF0EEA3F0758201124236022B91C2910F
:1026DA0090FC21E4F08D828E838FF012580A905B71
:1026EA005BC007C006C0051244E490FC1AE0F9A3D7
:1026FA00E0FA89828A83124541D005D006D0079034
:10270A00F7E9EDF0EEA3F0758201124236022B9141
:10271A0090FC21E0FABA06028061905B6BC007C0A8
:10272A0006C0051244E4D005D006D00790FC46E066
:10273A00FABA121B8D828E838FF074EC12580A90AB
:10274A00F7E9EDF0EEA3F0758201124236801F9090
:10275A00FC467417F08D828E838FF074EF12580A3C
:10276A0090F7E9EDF0EEA3F0758201124236C291BC
:10277A0012466890FC21E4F0022B9174012DF9E4D1
:10278A003EFA90F55CEBF089828A83C007C006C0E6
:10279A0005121732AC82D005D006D0078D828E83FF
:1027AA008FF0EC12580A8D828E838FF01259A1FB9A
:1027BA00EC603BBBFE028036905B74C007C006C06B
:1027CA00051244E4D005D006D0078D828E838FF09F
:1027DA001259A1F582C007C006C005124526C2914A
:1027EA00124668D005D006D00790FC21E4F090F795
:1027FA00E9EDF0EEA3F0758201124236022B918DBB
:10280A00828E838FF01259A1FB7C0090F586EBF043
:10281A00ECA3F0C374F09BE49C5019905A7F1244C5
:10282A00E490F7E97486F074F5A3F0758201124218
:10283A0036022B9190FC32E075F0F1A42472F974FF
:10284A00F335F0FA89828A83E06019905B81124439
:10285A00E490F7E97486F074F5A3F07582011242E8
:10286A0036022B918B0089828A83E8F090FC32E051
:10287A0075F0F1A42472F974F335F0FA09B900017C
:10288A000A890A8A0B750C0074012DF9E43EFA894B
:10289A00138A147515008B168C17850A82850B838B
:1028AA00850CF012576990FC32E0FC0C90FC32EC7B
:1028BA00F0BC0200400590FC32E4F090F7E974861F
:1028CA00F074F5A3F0758201124236022B918D82C3
:1028DA008E838FF01259A1FC7B0090FC26ECF0EB62
:1028EA00A3F090FC26E0F9A3E0FAC374709C740389
:1028FA009B402E74022DFBE43EFC8B138C14751541
:10290A000089168A1790F00075F00012576990F73F
:10291A00E97426F074FCA3F0758202124236022B87
:10292A009190F7E974A2F0745BA3F07582081242E1
:10293A0036022B9190FC26E0FBA3E090F7E97400A5
:10294A00F074F0A3F08B82124236022B91121A58BD
:10295A007B008B83121A1390FC2AE0FBA3E0FC9005
:10296A00F7E9EB2400F0EC34F0A3F075820112428F
:10297A0036022B918D828E838FF01259A1FC7B0037
:10298A008C828B83C007C006C0051214EAD005D01A
:10299A0006D00790F7E9EDF0EEA3F0758201124236
:1029AA0036022B91758200C007C006C00512156B4E
:1029BA00D005D006D00790F7E9EDF0EEA3F07582C6
:1029CA0001124236022B91C007C006C005121585B6
:1029DA00D005D006D00790F7E9EDF0EEA3F07582A6
:1029EA0001124236022B918D828E838FF01259A1E9
:1029FA00FC7B0090FC22ECF0EBA3F090F7E9EDF001
:102A0A00EEA3F0758201124236022B9190F7E97417
:102A1A0022F074FCA3F0758204124236022B918DC7
:102A2A00828E838FF0C007C006C0051244A3D0056A
:102A3A00D006D0078D828E838FF01259A1F582C0FD
:102A4A0007C006C005124526D005D006D0078D82DC
:102A5A008E838FF01259A1FC7B008C138B148B157B
:102A6A007516158B1790FC2175F000C007C006C0BB
:102A7A0005125769D005D006D00790F7E9EDF0EEB8
:102A8A00A3F0758215124236022B9190FC1DE0FBD1
:102A9A00A3E0FC90FC24EBF0ECA3F090F7E974219E
:102AAA00F074FCA3F0758215124236022B918D82C6
:102ABA008E838FF01259A1FC7B008C828B83C00716
:102ACA00C006C005121911D005D006D00790F7E943
:102ADA00EDF0EEA3F0758201124236022B9190FCC2
:102AEA0047E0F9A3E0FAA3E0A3E090FC2CE9F0EABE
:102AFA00A3F08D828E838FF01259A1FC90FC21F0F5
:102B0A0090FC21E0FBEC24FA404DEB2B2B902B1B85
:102B1A0073022B2D022B2D022B2D022B4F022B4F32
:102B2A00022B3EC007C006C005121585D005D00687
:102B3A00D0078023C007C006C0051219ECD005D003
:102B4A0006D0078012758200C007C006C00512159C
:102B5A006BD005D006D00790F7E9EDF0EEA3F0753B
:102B6A008201124236802090F7E97421F074FCA3A6
:102B7A00F0758201124236800E90F7E9EDF0EEA36D
:102B8A00F0758201124236900000222290F7D1E0BD
:102B9A00FFBF013990F7B1E0FEA3E0FF90F7D4E060
:102BAA00FCA3E0FD90F7B4E0FAA3E0FBEA4B601D5A
:102BBA008E828F83E0F9A3AE82AF838C828D83E904
:102BCA00F0A3AC82AD831ABAFF011B80DF90F7BA7B
:102BDA00E054FDF090DE11E0FF74084FF022AE825F
:102BEA00AF83E0FD20E703022CE18E828F83A3E00E
:102BFA00FD601DBD0102802ABD0202803BBD0302A9
:102C0A00805ABD04028076BDFE03022CA3022CE189
:102C1A0075370275380090FC4575F0001230EE02E7
:102C2A002CE190DE00E0FD7C007539288C3A8D821B
:102C3A008C83123162022CE18E828F83A3A3E0FC83
:102C4A00A3E0FD74062EF582E43FF583E0F539A38F
:102C5A00E0F53A8C828D83123162807B8E048F0577
:102C6A007B0074062EF582E43FF583E0F537A3E096
:102C7A00F5388C828D838BF01230EE805A90F7B142
:102C8A00E0FBA3E0FCA3E0FD753910753A008B82E6
:102C9A008C838DF0123162803E74022EFEE43FFF77
:102CAA007D00754BAA754C5B754D807513048D14A8
:102CBA008E828F838DF0125259E5828583F045F01A
:102CCA006012D29190012C12518DC29190012C1256
:102CDA00518D800375C9839000002290DF2FE4F0A4
:102CEA0090DF30F090DF31F090DF00740CF090DF6D
:102CFA0001744EF090DF0274FFF090DF037440F02D
:102D0A0090DF04E4F090DF05F090DF06F090DF0733
:102D1A007406F090DF08E4F090DF097424F090DF85
:102D2A000A743AF090DF0B74F1F090DF0C74CAF079
:102D3A0090DF0D74A3F090DF0E7401F090DF0F7432
:102D4A0023F090DF107411F090DF117436F090DFE9
:102D5A00127407F090DF13740FF090DF147418F0F8
:102D6A0090DF1514F090DF16746CF090DF1774037F
:102D7A00F090DF187440F090DF197491F090DF1A28
:102D8A007456F090DF1B7410F090DF1C74E9F09019
:102D9A00DF1D742AF090DF1EE4F090DF1F741FF02D
:102DAA0090DF237488F090DF247431F090DF25746B
:102DBA0009F090DF2E74C0F090DF07C4F090DF09AD
:102DCA007425F090DF0A7495F090DF0B7455F0903B
:102DDA00DF1A74B6F090DF1B7410F090DF1C74EAEF
:102DEA00F090DF1D742AF090DF1EE4F090DF1F746C
:102DFA001FF0221252DB025307122DFD12458B12CD
:102E0A0053341230B9124710121DD21230E8D2AF21
:102E1A00122F8CD29190000212518DC29190000A09
:0B2E2A0012518D124267121DF680F855
:105A040043616E6E6F742063616C6C207472616E9E
:105A1400736D69745F6C6F6E67207768696C65205D
:105A24004648535320486F7070696E67206F722028
:105A3400616C72656164792070726F6365737369F8
:105A44006E67207472616E736D69745F6C6F6E67DC
:105A540021004D41435F7478282920726574757262
:105A64006E6564206572726F72006E657665722071
:105A7400656E7465726564205458004648535378C3
:105A84006D6974206D65737361676520746F6F2031
:105A94006C6F6E67004648535320737461746520BD
:105AA400656E746572696E672053594E4348494E5A
:105AB400472066726F6D2077726F6E672073746112
:105AC40074650053594E43485F4D41535445522029
:105AD4002D3E2053594E43494E474D415354455250
:105AE4000046485353786D697420646F6E65006E88
:105AF4006574776F726B207061636B65742873795A
:105B04006E6329006E6574776F726B207061636BCE
:105B1400657428646973636F7665727929006372AA
:105B240061702C20706C6561736520757365204607
:105B3400485353786D6974282920696E73746561BC
:105B440064210064726F706F75742066696E616C95
:105B540020776169742100746F74616C20627974B8
:105B640065732074783A00756E64657272756E00A0
:105B7400627566666572206572726F72007374690D
:105B84006C6C2077616974696E67206F6E2074682D
:105B940065206C617374207061636B6574004E4F93
:0B5BA400204445414C005253544E0079
:102E3500AF827E017D0090DE0E7405F090FC457436
:102E450012F0EE7006ED7003022F827B107C279046
:102E5500DE11E0FA30E00D90FC467401F01BBBFF7B
:102E6500011C80EBEB4C7014D2919003E812518D4C
:102E7500C2919003E812518D90FFFF22BE01317E71
:102E85000090DE2A7440F0EFF0E532F0AB337C00C1
:102E9500EBF0E534F0C3E533943BE53494004008AA
:102EA5007B3B7C007D018021AB33AC347D008019F8
:102EB500C3E5339440E534940040087B407C007DB5
:102EC500018006AB33AC347D007480252942D6855C
:102ED5002682852783A935AA368A00E8F0852682C9
:102EE500852783A3E9F0852682852783A3A374DE3E
:102EF500F0852682852783A3A3A3742AF0852682DD
:102F0500852783A3A3A3A3A3EBFAF08526828527B0
:102F150083A3A3A3A3E054E0F0852682852783A39A
:102F2500A3A3A3A3A3A3E0543F4440F08526828531
:102F35002783A3A3A3A3A3A3A3E054CFF0E529422A
:102F4500D6E52942D7E52955D160FAE529F452D1CC
:102F550090DE0E7405F090DE11E0FA74014AF0E59A
:102F650033C39BF533E5349CF534EB2535F535EC6A
:102F75003536F53690FC457413F0022E4790FC4526
:102F85007414F090000022E522700512426780F764
:102F950022AFBE747F5FF5BE43BE8090DE0B74F733
:102FA500F090DE0774FFF090DE09F0438C10AF8CD3
:102FB50074FE5FF58CD2BD439A02758900C2C57552
:102FC5008B00C2E843A90243B9028526828527837F
:102FD500A3A3A3A3E054E0F0852682852783A3A3BA
:102FE500A3A3A3A3E0549F4420F0852682852783CD
:102FF500A3A3A3A3A3A3A3E04408F0852682852762
:1030050083A3A3A3A3A3A3A3E054FC4401F090DEF0
:1030150001E0FF74FE5FF0E4F525F523F524F522C4
:1030250090DE0EF090DE107404F090DE13F090F751
:10303500BBE4F090F7BAF090F7AFF0A3F090F7B1DA
:103045007488F074F5A3F0E4A3F090F7B4F0A3F05E
:1030550090F7B6F090F7B7F090F7B8F0A3F090DEE0
:103065000E7405F090DE107408F090DE13F090DE1B
:1030750012E0FF74014FF090DE15E0FF74014FF090
:1030850090F7CDE4F090F7CCF090F7C1F0A3F09075
:10309500F7C374A8F074F5A3F0E4A3F090F7C6F0B5
:1030A500A3F090F7C8F090F7C9F090F7CAF0A3F035
:1030B500439A02221245B58582288528F005F074C9
:1030C50001800225E0D5F0FBF529E52875F008A477
:1030D50024F9F52674F735F0F52790FC457402F0D0
:1030E500022F96D29022C29022AFF0AE83E5829055
:1030F500F7D6F0EEA3F0EFA3F090F7BBE06034D283
:10310500919003E812518DC2919003E812518DD22E
:10311500919003E812518DC2919003E812518DD21E
:10312500919003E812518DC2919003E812518D9050
:10313500FFFF2290F7D6E0FDA3E0FEA3E0FF90F7A6
:10314500ACEDF0EEA3F0EFA3F090F7AFE537F0E5C7
:1031550038A3F090F7BB7401F090000022AF83E52F
:103165008290F7D9F0EFA3F090F7BBE06034D291ED
:103175009003E812518DC2919003E812518DD291BE
:103185009003E812518DC2919003E812518DD291AE
:103195009003E812518DC2919003E812518D90FF72
:1031A500FF2290F7D9E0FEA3E0FF7D0090F7ACEE9B
:1031B500F0EFA3F0EDA3F090F7AFE539F0E53AA312
:1031C500F090F7BB7401F0900000227F007E029022
:1031D500DE0EE4F090F7AFE0FCA3E0FDC3EC942035
:1031E500ED940040047B2080068C037F017E0A8BD2
:1031F500017A00ECC399FCED9AFD90F7AFECF0ED88
:10320500A3F08B05ED603690F7ACE0FAA3E0FBA3E5
:10321500E0FC8A828B838CF01259A190DE20F0901D
:10322500F7ACE0FAA3E0FBA3E0FC0ABA00010B90BF
:10323500F7ACEAF0EBA3F0ECA3F01D80C790DE112C
:10324500E0FD4EF0EF600590F7BBE4F02290F7BB90
:103255007402F07582002290F7B1E0FDA3E0FEA3B1
:10326500E0FF90DE11E0FCB40100E433FC20E0F265
:1032750090DE0EE4F090DE16E0FC7B0090F7B4ECF7
:10328500F0EBA3F090F7BAE0FC30E11390F7BB74D4
:1032950003F090DE11E0FC74044CF090FFFF2290E7
:1032A500F7BAE04402F090F7B4E0FBA3E0FCC37486
:1032B500209BE49C501CD29190012CC007C006C0F5
:1032C5000512518DC29190012C12518DD005D00659
:1032D500D00790F7B4E0FBA3E0FC8D07EB4C60163C
:1032E50090DE20E0FD8F828E83F0A3AF82AE831B3C
:1032F500BBFF011C80E6E52C452D6009852C8285E8
:103305002D8312148990F7B4E0FEA3E0FFC3EE9479
:1033150020EF9400501DE52A452B6009852A8285FA
:103325002B8312148990DE11E0FF74084FF090F79B
:10333500BBE4F090DE11E0FF74404FF090F7B4E08D
:10334500FEA3E08E82F5832285822E85832F22853A
:1033550082308583312275370175380090002575D7
:10336500F0400230EEAFF0AE83E58290F7DBF0EE91
:10337500A3F0EFA3F090F7DBE0FDA3E0FEA3E0FFF1
:1033850074022DFDE43EFE8D828E838FF01259A1CD
:10339500FDA31259A18D2575220122AF827DEB7EF9
:1033A5005BBF030874EEB513037513048D828E831A
:1033B500A3E090F7DEF0AC1390F7DEE0FBBBFF0275
:1033C500803EEBB50723EC700890F7DE74FFF080C4
:1033D500E71C8D828E83E02DFDE43EFE8D828E837B
:1033E500A3E0FB90F7DEF080CF8D828E83E02DFD8C
:1033F500E43EFE8D828E83A3E0FB90F7DEF080B87D
:103405008D828E8322AFF0AE83E58290F7DFF0EEFA
:10341500A3F0EFA3F090F7DFE0F53DA3E0F53EA3C1
:10342500E0F53F7402253DFAE4353EFBAC3F8A8268
:103435008B838CF01259A1F8A31259A1F9893B7518
:103445003C007402B53B06E4B53C0280227407B526
:103455003B06E4B53C028002804274AF58FE7F0013
:103465008A828B838CF0EE12580AA3EF12580A8ACF
:10347500828B838CF01259A1FAA31259A1F5828A85
:10348500131233A0AE82AF8390F7E2EEF0EFA3F014
:103495008E828F83A3A3E0FE7F00801C8982881320
:1034A5001233A0AC82AD8390F7E2ECF0EDA3F08C83
:1034B500828D83E0FCFE7F007406253DFBE4353EEE
:1034C500FCAD3F8B828C838DF01259A1FCA3125960
:1034D500A1FDC3EC9EED9F50048C068D07EE4F7049
:1034E5000990DE11E0FD74204DF090F7E2E0FCA3B9
:1034F500E0FD8E398F3A8C828D8302316290DE0E2B
:10350500E4F090DE11E0FF30E40E90F7BBE4F090BC
:10351500DE11E0FE74804EF0EF30E22490DE11E41F
:10352500F090FC467404F090F7BBE4F0D291900063
:1035350014C00712518DC29190001412518DD007FD
:1035450090F7BBE0FEBE0319D291900032C007127E
:10355500518DC29190003212518DD00790F7BBE486
:10356500F090F7BBE06003023842EF20E003023839
:103575004290DE0EE4F090DE16E0FFFE7B407C001C
:103585007D40EE601690DE20E0FA8B828C838DF014
:1035950012580AA3AB82AC831E80E7E540FE20E704
:1035A5000302371574605EFD6015BD20030236CF3A
:1035B500BD40030236DBBD600302370002382A74C2
:1035C5001F5EFF7041AD41BD0002801CBD0602803B
:1035D50005BD0826800C90004075F04012340A02A3
:1035E500382A12335B02382A753702753800905B2A
:1035F500C975F0801230EE02382A90004075F0400F
:103605001244A202382ABF0145AD41BD0002800522
:10361500BD0A268012753702753800905BC975F0B2
:10362500801230EE02382A753701753800905BCC70
:1036350075F0801230EE02382A90DE11E0FD74201C
:103645004DF090004075F0401244A202382ABF02A6
:1036550036AD41BD00028008BD120302382A801232
:10366500753702753800905BC975F0801230EE022F
:10367500382A90DE11E0FD74204DF090004075F081
:10368500401244A202382ABF032BE4B54112753714
:1036950002753800905BC975F0801230EE02382A49
:1036A50090DE11E0FD74204DF090004075F0401261
:1036B50044A202382A90004075F0401244A290DEE0
:1036C50011E0FD74204DF002382A90DE11E0FD7402
:1036D500204DF002382AE52E452F60131236E6807C
:1036E5000BC02EC02F90004075F0402202382A9062
:1036F500004075F04012385902382A90DE11E0FD7D
:1037050074204DF090004075F0401244A202382A12
:1037150074605EFD6015BD20030237E1BD40030204
:1037250037F5BD600302381802382A741F5EFF7032
:1037350048AE41BE010302382ABE030302382ABE41
:103745000502800BBE070302382ABE0917800990BF
:10375500DE00E542F002382A90004075F040123351
:103765006A02382A90004075F0401244A290DE119A
:10377500E0FE74204EF002382ABF0129AE41BE0199
:103785000302382ABE030302382ABE110302382A6F
:1037950090004075F0401244A290DE11E0FE7420C6
:1037A5004EF002382ABF0220AF41BF01028076BF2A
:1037B5000302807190004075F0401244A290DE1122
:1037C500E0FF74204FF0805D90DE11E0FF74204F24
:1037D500F090004075F0401244A280499000407579
:1037E500F0401244A290DE11E0FF74204FF08035C6
:1037F500E52E452F6012123800800BC02EC02F9089
:10380500004075F04022801D90004075F040123850
:1038150059801290DE11E0FF74204FF09000407542
:10382500F0401244A290DE11E0FF74404FF0E546EF
:103835004547700990DE11E0FF74084FF090F7BB23
:10384500E0FFBF01031231D090F7BBE0FFBF0203D9
:1038550002325C22AFF0AE83E58290F7E4F0EEA38E
:10386500F0EFA3F090F7E4E0FDA3E0FEA3E0FF8D09
:10387500828E838FF01259A1FC20E703023A7474FB
:10388500012DFAE43EFB8F048A828B838CF012595A
:10389500A1FC6025BC01028032BC02028043BC034E
:1038A50003023922BC0403023957BCFD03023974F3
:1038B500BCFE03023A2E023ADA75370275380090DB
:1038C500FC4575F0001230EE023ADA90DE00E0FCBD
:1038D5007B007539288B3A8C828B83123162023AD0
:1038E500DA74022DFAE43EFB8F048A828B838CF016
:1038F5001259A1FAA31259A1FB74062DF8E43EF959
:103905008F04888289838CF01259A1F539A3125945
:10391500A1F53A8A828B83123162023ADA8D028EE0
:10392500038F048A488B498C4A74062DF8E43EF9C6
:103935008F04888289838CF01259A1F537A3125917
:10394500A1F538854882854983854AF01230EE0213
:103955003ADA90F7B1E0FAA3E0FBA3E0FC75391081
:10396500753A008A828B838CF0123162023ADA74DE
:10397500042DFAE43EFB8F048A828B838CF0125966
:10398500A1F8A31259A1F9B80477B90074746C446D
:103995005C606EC002C003C00474062DF8E43EF9F5
:1039A5008F04888289838CF01259A1F548A3125996
:1039B500A1F549905C6CE493FC8C4B754C00C3E518
:1039C5004B9548E54C9549D004D003D002501A8553
:1039D5004B39854C3A905C6CC004C003C00212316F
:1039E50062D002D003D004801885483985493A90C1
:1039F5005C6CC004C003C002123162D002D003D097
:103A0500048A828B838CF01259A1FAA31259A1FB67
:103A1500BA0505BB00028003023ADAE4F539F53A46
:103A2500900000123162023ADA74022DFAE43EFB8C
:103A35008F0490FC4B74CEF0745BA3F07480A3F0FC
:103A45007513047514008A828B838CF0125259E524
:103A5500828583F045F06012D29190012C12518D30
:103A6500C29190012C12518D806B75C9838066902F
:103A7500F7D1E0FCBC015674022DFDE43EFE8D82BB
:103A85008E838FF01259A1FDA31259A1FE90DE0E6F
:103A9500E4F090DE16E0FF7C007512088F828C83BF
:103AA500C007C006C005C0041251D9D004D005D046
:103AB50006D007EF4C601690DE20E0FB8D828E83EA
:103AC500F0A3AD82AE831FBFFF011C80E690F7BA5D
:103AD500E054FDFFF09000002290F7CCE0FF30E1CC
:103AE5000A90FC467405F090FFFF2290DE0E7405E7
:103AF500F090DE16E0FF8F4D754E0090DE17E0FC6E
:103B0500E4254DF54DEC354EF54E90F7CAE0FCA396
:103B1500E0FD4C705890F7C6E4F0A3F090DE2AE083
:103B250090F7C8F090DE2AE090F7C9F090DE2AE021
:103B3500FD7C0090F7CAEDF0ECA3F090DE2AE0FAE8
:103B4500E4FB2DFDEA3CFC90F7CAEDF0ECA3F0E5B3
:103B55004D24FCF54DE54E34FFF54EC374049D74BC
:103B6500029C500990F7CA7404F003A3F0E52955A7
:103B7500D16012D29190001412518DC2919000140F
:103B850012518D80E890F7C3E0FBA3E0FCA3E09021
:103B9500F7C6E0FAA3E0FFEA2BFBEF3CFC748025B7
:103BA5002942D685268285278374DEF0852682857F
:103BB5002783A3742AF0852682852783A3A38C07F0
:103BC500EFF0852682852783A3A3A3EBF0852682C4
:103BD500852783A3A3A3A3A3A3A3E0543FF085262E
:103BE50082852783A3A3A3A3A3A3A3E054CF441053
:103BF500F074052526FEE43527FF90DE16E0FD8EE0
:103C0500828F83EDF074042526FEE43527FF90DED0
:103C150017E08E828F83541FF5F0E054E045F0F0F5
:103C250090F7C6E0FEA3E0FFEE254DFCEF354EFD17
:103C3500C374049C74029D500B7404C39EF54D74AB
:103C4500029FF54EC37440954DE4954E502890FC67
:103C5500467406F090DE14E0FD74FE5DF075120406
:103C65009000051251D9751210854D82854E83122B
:103C750051D990FFFE22E52942D6E52942D7E54DE7
:103C85002EFEE54E3FFF90F7C6EEF0EFA3F0E529D7
:103C950055D160FAE529F452D190F7C6E0FEA3E0CC
:103CA500FF90F7CAE0FCA3E0FDC3EE9CEF9D402C1E
:103CB50090F7CCE04402F090F7CAE4F0A3F090DE70
:103CC5000E7405F0AE2374BF5524FF8E238F249008
:103CD500DE14E0FF74FE5FF09000012290DE0E74AA
:103CE50005F0AE2374BF5524FF8E238F2490DE1478
:103CF500E0FF74FE5FF09000002290F7CCE0FF201B
:103D0500E1012290F7C3E0FDA3E0FEA3E0FF90F7F9
:103D1500E7EDF0EEA3F090F7C8E0F55674FFB55661
:103D250002800302420E90F7C9E0FBBB80005003FE
:103D35000241F0EB246C50030241F0EB2480FA249D
:103D45000A83F582EA241883F583E473790EA4E1E6
:103D5500C1F819306952F0F0F0F0D104647EF0A397
:103D65003D3E3F3F3E3F4040404041414141404153
:103D7500414141418D828E838FF01259A1FA740120
:103D85002DF551E43EF5528A5475550090F7CAE574
:103D950054F0E555A3F0855182855283E0F55374BF
:103DA500012551F556E43552F557A9538902E4F931
:103DB5002554F554EA3555F55590F7CAE554F0E51F
:103DC50055A3F0855682855783E0F8855182855243
:103DD50083A3A3884F8950E0FAE4254FF54FEA35D0
:103DE50050F550854F3585503690F7C8E0FA90F775
:103DF500C9E0F5328554338555348A82122E3590C3
:103E0500F7CAE4F0A3F00242068D828E838FF0128A
:103E150059A1FA8D828E83A38A4F755000E0FA74FA
:103E2500022DF556E43EF5578A018902E4254FF542
:103E35004FEA3550F550A84FAA5090F7CEE8F0EA72
:103E4500A3F090F7C6E0F9A3E0FAE924FEF54FEAFE
:103E550034FFF550854F54855055E5544555603D23
:103E650090F7CEE0F551A3E0F55274012551F9E440
:103E75003552FA90F7CEE9F0EAA3F08556828557D8
:103E850083E0FAA3858256858357855182855283BF
:103E9500EAF0155474FFB55402155580BD90F7C866
:103EA500E0FA90F7C9E0F5327535CA7536F775331E
:103EB500027534008A82122E3502420690F7CCE054
:103EC500FA20E23C8D828E838FF01259A1FA8D8201
:103ED5008E83A38A4F755000E0FA90F7E774022DA0
:103EE500F0E43EA3F08A018902E4F9254FF54FEA93
:103EF5003550F550A84FAA5090F7CEE8F0EAA3F058
:103F050090F7CAE0F9A3E0FA894F8A50C374409547
:103F15004FE495505006754F40755000E9C3954FD5
:103F2500F9EA9550FA90F7CAE9F0EAA3F090F7E7B5
:103F3500E0F554A3E0F555854F56855057E55645B0
:103F450057603D90F7CEE0F551A3E0F55274012599
:103F550051F9E43552FA90F7CEE9F0EAA3F0855429
:103F650082855583E0FAA3858254858355855182E0
:103F7500855283EAF0155674FFB55602155780BD74
:103F850090F7C8E0FA90F7C9E0F5327535CA75368D
:103F9500F77533027534008A82122E35024206D235
:103FA50091900002C007C006C00512518DC29190C4
:103FB500000212518DD005D006D00790F7C8E0FA5F
:103FC50090F7C9E0F53290F7C6E0F533A3E0F53494
:103FD5008D358E368A82122E350242067535D37599
:103FE500365B8B3275330D753400855682122E354E
:103FF50002420690FC47E0F8A3E0F9A3E0A3E088BD
:104005003589368B32753304753400855682122E08
:10401500350242067535B875365B8B3275331175C9
:104025003400855682122E3502420690F7C6E0F519
:1040350033A3E0F5348B328D358E36855682122EBC
:10404500359000C812518D1245C40242067535AF30
:1040550075365B8B32753309753400855682122EA1
:10406500350242068D828E838FF01259A1FC7401B0
:104075002DF9E43EFABC0202800ABC03028021BC91
:104085000429800DC002C00112468DD001D00280E6
:104095001AC291C002C0011246D7D001D002800BCE
:1040A500C002C0011246AED001D00290F7C8E0FCB4
:1040B50090F7C9E0F53290F7C6E0F533A3E0F534A3
:1040C50089358A368C82122E3502420690F7CA74DB
:1040D50001F0E4A3F07535367536DF90F7C8E0FCDE
:1040E50090F7C9E0F53290F7CAE0F533A3E0F5346F
:1040F5008C82122E3590F7CAE4F0A3F00242068DA9
:10410500028E048C017C0090FC4B74E1F0745BA37F
:10411500F07480A3F07513098C148A8289838CF05E
:10412500C007C006C005125259E5828583F0D00547
:10413500D006D00745F0600302420675C98090F7A6
:10414500C8E0FC90F7C9E0F53290F7C6E0F533A377
:10415500E0F5348D358E368C82122E35024206906E
:10416500FC45E4F090FC46F090F7E9EDF0EEA3F0A5
:1041750075820212423602420690F7CAE4F0A3F0B5
:1041850090F7C8E0FC90F7C9E0F532753310753447
:10419500007535F07536138C82122E3580638D824D
:1041A5008E838FF01259A1FC74012DF9E43EFABCFF
:1041B5000002800BBC010F90FC8E7401F0800C9006
:1041C500FC8EE4F0800590FC8EE4F090F7C8E0FCEE
:1041D50090F7C9E0F53290F7C6E0F533A3E0F53482
:1041E50089358A368C82122E35801690F7C6E0F511
:1041F50033A3E0F5348B328D358E36855682122EFB
:104205003590F7CCE054FDF022E530453160198555
:104215003082853183121489AE82AF83EE4F7010E0
:1042250090F7CCE054FDF02290F7CCE054FDFFF080
:1042350022E58290F7EBF090F7CCE054FDF090F793
:10424500C8E0FF90F7C9E0F53290F7EBE0FE8E335A
:1042550075340090F7E9E0F535A3E0F5368F820275
:104265002E35E52330E01175220274FE5523FEAF8D
:10427500248E238F2443BE01E5235406602F90FC32
:1042850045740AF075220374FD5523FEAF248E2371
:104295008F2490DE01E0FF74044FF0900008125166
:1042A5008D90DE01E0FF74FB5FF075220190DE0E5C
:1042B500E4F090DE11E0FF30E21A90DE11E0FF74C9
:1042C500DB5FF090F7AFE4F0A3F090F7B4F0A3F064
:1042D50090F7BBF090DE0E7405F090DE11E0FF3034
:1042E500E52090DE11E0FF74CF5FF090FC46740886
:1042F500F090F7C1E4F0A3F090F7C6F0A3F090F7C3
:10430500CDF090DE14E0FF30E62090DE14E0FF747F
:104315009F5FF090FC467408F090F7C1E4F0A3F0BD
:1043250090F7C6F0A3F090F7CDF0E52320E20574F1
:1043350004B52214122F9690FC45740BF074FB55AE
:1043450023FEAF248E238F24E52330E4111235029A
:1043550074E75523FE740F5524FF8E238F24E5241F
:1043650030E65490FC45740CF0123ADEAE82AF8311
:10437500BEFE41BFFF3E90F7EC7406F0E4A3F0905B
:10438500F7C8E0FF90F7C9E0F5327535EC7536F7FB
:104395007533027534008F82122E3590F7C8E0FF11
:1043A5007535EC7536F77532017533027534008F46
:1043B50082122E35123CFFE52354E07006E52454A5
:1043C500BD602990FC467409F075120890004412EE
:1043D50051D98523828524837512101251D974E031
:1043E5005523FE74BD5524FF8E238F2422C0E0C0C3
:1043F50082C083C007C006C005C004C0D075D00008
:10440500E5BE30E6FB90DE06E0FF7E00E5234207D1
:10441500E52442068F238E2490DE02E0FDE4CDC420
:10442500CD6DCD54F0CD6DFCED4207EC42068F23EA
:104435008E2490DE04E025E0FCE4FD4207EC420614
:104445008F23EEF52430E11290F7CCE054FEF0AE68
:104455002374FD5524FF8E238F24758B00C2E8D06D
:10446500D0D004D005D006D007D083D082D0E0329A
:10447500C0E0C007C0D075D000E5BE30E6FBC2AFD6
:10448500E58930E703752203AFBE74FC5FF5BE75A1
:0E4495008900C2C5D2AFD0D0D007D0E032220D
:105BAF00534443437633353000444F4E53444F4EA6
:105BBF00474C45207230363036000000000000524E
:105BCF0053544E00554E494D504C454D454E54453E
:105BDF00440052455345545F4E4F57001201000287
:105BEF0000000020501D48600101010203010A0658
:105BFF0000020000002001000902200001010080C6
:105C0F00FA0904000002FFFFFF00070585024000AC
:105C1F000107050502400001040309040C035200AB
:105C2F006600430061007400180344006F006E00AB
:105C3F007300200044006F006E0067006C00650069
:105C4F000A03300030003900610012034D00530089
:105C5F0046005400310030003000FD00FF280000E6
:105C6F0000000104000100000000000000000157C7
:105C7F00494E555342000000000000000000000094
:055C8F00000000000010
:1044A300AF83E58290F7EEF0EFA3F090F7EEE0FE36
:1044B300A3E0FF7C007D008E028F038A828B83E062
:1044C300F9A3AA82AB83E960070CBC00EE0D80EB75
:1044D3007532F08C338D348E358F367582FE022E15
:1044E30035AF83E58290F7F0F0EFA3F090F7F0E0BB
:1044F300FEA3E0FF7C007D008E028F038A828B8304
:10450300E493F9A3AA82AB83E960070CBC00ED0D29
:1045130080EA8E358F367532F08C338D347582FE9A
:10452300022E35E58290F7F2F07535F27536F775A0
:1045330032F17533017534007582FE022E35AF8377
:10454300E58290F7F3F0EFA3F07535F37536F77561
:1045530032F27533027534007582FE022E35AF8256
:10456300AE83ADF0FC90F7F5EFF0EEA3F0EDA3F022
:10457300ECA3F07535F57536F77532F375330475BD
:0845830034007582FE022E35A2
:0314E400750D0083
:10458B007EF97FF78FD57EF97FF78ED47E017FF88A
:10459B008FD37E017FF87F008ED28F137514188F07
:1045AB001590F7F975F00002574A7403B50D0475B1
:1045BB0082FF22850D82050D2290DF46E0FFBFF0C2
:1045CB000E90DF47E0FFBF0D0690DF487469F0C225
:1045DB00AF759A0075B80075A8001230EBAFBE74BA
:1045EB007F5FF5BE75D69FC291020000221257BEA7
:1045FB00AC82AD83AEF0FFC004C005C006C007900F
:10460B0037BD75F086743D125646AC82AD83AEF065
:10461B00FFE58124FCF581E4C0E0C0E074C0C0E09C
:10462B007441C0E08C828D838EF0EF1258DEAC8229
:10463B00AD83AEF0FFE58124FCF5818C828D838EFA
:10464B00F0EF1257D1AC82AD83AEF090DF09EEF0F4
:10465B008D0390DF0AEBF090DF0BECF02275E10499
:10466B0090DF3BE0FFBF01F890FC1CE0F5E190FC14
:10467B001CE0FFBF04012290DF3BE0FFBF01028083
:10468B00ED2290FC1CE0FFBF02012290DF13E0FF44
:10469B0074F05FF0E0FF740F4FF090FC1C7402F0AD
:1046AB00024B0D90FC1CE0FFBF03012290DF13E0D7
:1046BB00FF74F05FF0E0FF740A4FF090FC1C740382
:1046CB00F0F5E190DF3BE0FFBF13F82290FC1CE01C
:1046DB00FFBF04012290DF13E0FF74F05FF0AF9196
:1046EB0074EF5FF59175E10490DF3BE0FFBF01F8DC
:1046FB00AF9B74FC5FF59BAFE974EF5FF5E990FC42
:10470B001C7404F02290FC1FE4F0A3F090FC12F058
:10471B00A3F090FC14F0A3F053C6C7759D00859EC3
:10472B009E439E0485A9A943B90190FC1C7404F017
:10473B00751300751400F51590F81275F0001257EB
:10474B004A122CE5D2A87591D175E900750E00437C
:10475B009A0175E10490DF3BE0FFBF01F8227E0078
:10476B007F00C3EE94DCEF9405502490DF3CE0FD1A
:10477B005450600490000122900032C007C0061212
:10478B0051BBD006D00774322EFEE43FFF80D3908E
:10479B00000022AF83E58290FC3CF0EFA3F090FC8D
:1047AB003EE4F090DF02E0FF90DF3BE0FEBE131E25
:1047BB00A291B3920190FC8EE0FEA201E43352066B
:1047CB00EE24FF9291C007124267D00780DAC291A4
:1047DB0090FC8AE4F090FC38E0FDA3E0FE90FC80B6
:1047EB00EDF0EEA3F090FC3AE0FBA3E0FC90FC862E
:1047FB00EBF0ECA3F090FC36E0F9A3E0FA90FC822E
:10480B00E9F0EAA3F090FC84E9C39BF0EA9CA3F0E7
:10481B0090FC84E0FBA3E0FC8D138E148B828C83C5
:10482B00C007C006C005C002C001125825AB82AC40
:10483B0083D001D002D005D006D00790FC88EB299D
:10484B00F0EC3AA3F0E94A705D90FC3CE0FBA3E08E
:10485B00FC8B828C83E0F8880F75100090FC36E59A
:10486B000FF0E510A3F090DF04E0F8530003B8005D
:10487B00028018B80102800302494390FC36740190
:10488B00250FF0E43510A3F002494390FC3C740172
:10489B002BF0E43CA3F090FC36E0FBA3E0FC90DFB4
:1048AB0002EBF002494390DF04E0FC530403BC002D
:1048BB00028046BC0102800302494390FC3CE0FBB2
:1048CB00A3E0FC90FC3FE9F0EAA3F090FC417401FB
:1048DB00F0E4A3F08B828C83C007C002C00112519D
:1048EB0038D001D002D00790FC3CE0FBA3E0FC8960
:1048FB00008B828C83E8F0803FED4E603690FC8815
:10490B00E0FDA3E090DF02EDF090DF04E0FE74FC2D
:10491B005EF090FC88E0FDA3E0FEC374FF9DE49E77
:10492B00500990DF04E0FE74024EF090FC8A740193
:10493B00F0800590DF02E9F0D2A890FC8BE0FE201E
:10494B00E303024A7190DF04E0FE530603BE010647
:10495B0090FC3E7401F090FC3EE0FE90FC3CE0FCD1
:10496B00A3E0FDEE2CFAE43DFB90FC36E0F8A3E06F
:10497B00F990FC5DE8F0E9A3F08A828B83C007C055
:10498B0006C005C004125487AA82AB83D004D0059D
:10499B00D006D00790FC8BE0F9530104B90448C052
:1049AB0007EE2CF8E43DF990FC8BE0FF5307F090F9
:1049BB00FC61E8F0E9A3F090FC63EAF0EBA3F09064
:1049CB00FC65EFF088828983C007C006C005C00470
:1049DB00C003C0021254C1D002D003D004D005D002
:1049EB0006D007D0078046C007EE2CF8E43DF990BF
:1049FB00FC8BE0FF5307F090FC68E8F0E9A3F09024
:104A0B00FC6AEAF0EBA3F090FC6CEFF088828983F0
:104A1B00C007C006C005C004C003C00212550AD0AF
:104A2B0002D003D004D005D006D007D007EE601E0D
:104A3B0090FC8BE0FE5306F0BE50098C828D837484
:104A4B0010F080228A068C828D83EEF0801890FC09
:104A5B008BE0FE5306F0BE500890DF027410F0801E
:104A6B000590DF02EAF090FC3CE0FDA3E0FE90FC39
:104A7B0018EDF0EEA3F090FC7EE4F0A3F075E103EB
:104A8B007D607EEA90DF3BE0FCBC1302802F1DBDF6
:104A9B00FF011EED4E6026A291B3920190FC8EE0B9
:104AAB00FCA201E4335204EC24FF9291C007C00630
:104ABB00C005124267D005D006D00780C790FC8E88
:104ACB00E0FC1392019291ED4E700690FC4674132C
:104ADB00F090DF3BE0FEBE131EA291B3920190FC5F
:104AEB008EE0FEA201E4335206EE24FF9291C00742
:104AFB00124267D00780DAC29190DF02EFF0758225
:104B0B000122D2A875130075140075150290F812C6
:104B1B0075F00012574A90FC12E4F0A3F090FC14CD
:104B2B00F0A3F090FC16F090FC1704F090F811E451
:104B3B00F0AF9B74FC5FF59BAFE974EF5FF5E97524
:104B4B00E10290DF3BE0FFBF0DF84391102290FC98
:104B5B008D7401F02290FC8DE4F022C021C0E0C0E6
:104B6B00F0C082C083C007C006C005C004C003C02C
:104B7B0002C001C000C0D075D00090FC457411F08C
:104B8B00C28990DF3BE0FFBF0D028003024CB8905F
:104B9B00FC8EE0FF139202929190FC77E0E0602A8A
:104BAB0090FC78E0FEA3E0FF90FC78E024FFFCA3F0
:104BBB00E034FFFD90FC78ECF0EDA3F074FF2F4098
:104BCB000990DF04E0FF74FC5FF090FC1C7402F0B2
:104BDB0090F811E025E0FEE42412FFEE34F8FEE03D
:104BEB0075F002A42412FC74FC35F0FD8C828D83CD
:104BFB00E0FAA3E0FB74012AF8E43BF98C828D8385
:104C0B00E8F0E9A3F0EA2FF582EB3EF583E5D9F066
:104C1B0090F811E075F002A42412F58274FC35F0C3
:104C2B00F583E0FEA3E0FFC39402501A90F811E065
:104C3B0075F002A42412F58274FC35F0F583E0FEC6
:104C4B00A3E0FF4E701A90F811E0FF75F002A42458
:104C5B0012F58274FC35F0F58374FFF07401A3F048
:104C6B0090FC78E0A3E090FC78E0F5F0A3E045F051
:104C7B006003024E7590FC77E0E07003024E759076
:104C8B00FC7AE0FEA3E0FF90FC78EEF0EFA3F0904F
:104C9B00FC78E0FEA3E090DF02EEF090DF04E0FF93
:104CAB0074FC5FF0E0FF74024FF0024E7590DF3B37
:104CBB00E0FFBF13028003024E7590FC8AE0E070A8
:104CCB0003024E0690FC2EE0FEA3E0FF0EBE000199
:104CDB000F90FC2EEEF0EFA3F090FC7EE0FEA3E035
:104CEB00FF90FC82E0FCA3E0FDEEB50406EFB505FA
:104CFB00028003024DD990FC80E0A3E090FC80E0A1
:104D0B00F5F0A3E045F0603790FC80E0FEA3E0FFF8
:104D1B00BEFF05BF0002801490FC80E024FFFEA3C1
:104D2B00E034FFFF90FC80EEF0EFA3F090FC86E008
:104D3B00FEA3E0FF90FC7EEEF0EFA3F0024DD990C6
:104D4B00FC82E0F513A3E0F51490FC7CE0FF7E0001
:104D5B008F828E83125825AE82AF8390FC18E0FCB5
:104D6B00A3E0FDEE2CF582EF3DF583E4F090FC7CA7
:104D7B00E02401F0E0FF90FC7DE0FEEFB50605902E
:104D8B00FC7CE4F090FC82E0F513A3E0F51490FCBE
:104D9B007CE0FF7E008F828E83125825AE82AF831C
:104DAB0090FC18E0FCA3E0FDEE2CFEEF3DFF8E82A5
:104DBB008F83E0701090FC21E4F090FC467412F0AD
:104DCB00124668C29190FC7E7401F0E4A3F090FC53
:104DDB0088E0FEA3E0FF90FC88E024FFFCA3E03416
:104DEB00FFFD90FC88ECF0EDA3F0BEFF22BF001F8F
:104DFB0090DF04E0FF74FC5FF0801490FC88E024EB
:104E0B00FFFEA3E034FFFF90FC88EEF0EFA3F090E1
:104E1B00FC1C7403F090FC82E0F513A3E0F51490F6
:104E2B00FC7CE0FF7E008F828E83125825AE82AF12
:104E3B008390FC7EE0FCA3E0FD90FC7EE02401F07F
:104E4B00A3E03400F0EC2EFEED3FFF90FC18E0FCED
:104E5B00A3E0FDEE2CF582EF3DF583E0F5D990FC58
:104E6B001AE02401F0A3E03400F0D0D0D000D00140
:104E7B00D002D003D004D005D006D007D083D08287
:104E8B00D0F0D0E0D02132C021C0E0C0F0C082C051
:104E9B0083C007C006C005C004C003C002C001C068
:104EAB0000C0D075D00075110090FC457410F0AEA9
:104EBB009B74FC5EF59BE5E9420EE5E930E0209042
:104ECB00FC1DE0FDA3E08D067D00AB9C7C0090FCFF
:104EDB001FED4BF0EE4CA3F0AEE974FE5EF5E9E589
:104EEB00E95470700302509B90FC1CE0FEBE030A59
:104EFB00AE0E748F5EF50E02509490F811E0FEB476
:104F0B000100E4332416F582E434FCF583E0FEBEA5
:104F1B000102800302504B90FC8BE0FE20E1030268
:104F2B00502490DF04E0FE530603BE01037511010C
:104F3B0090FC8BE0FE530601BE017090F811E0254A
:104F4B00E0FDE42412FEED34F8FDAB117C00EB2EFA
:104F5B00FEEC3DFDE0F929FAE42412F9EA34F8FA03
:104F6B00EB29FBEC3AFCE075F002A42412F58274F9
:104F7B00FC35F0F583E0F9A3E0FAA8117F00E9C353
:104F8B0098F9EA9FFA90FC8BE0FF5307F090FC61D5
:104F9B00EBF0ECA3F090FC63E9F0EAA3F090FC6576
:104FAB00EFF08E828D831254C1806E90F811E02544
:104FBB00E0FEE42412FFEE34F8FEAC117D00EC2F82
:104FCB00FFED3EFEE025E0FAE42412FBEA34F8FAAA
:104FDB00EC2BFCED3AFDE075F002A42412F5827483
:104FEB00FC35F0F583E0FAA3E0FBA8117900EAC3E6
:104FFB0098FAEB99FB90FC8BE0F95301F090FC686D
:10500B00ECF0EDA3F090FC6AEAF0EBA3F090FC6CF3
:10501B00E9F08F828E8312550A90F811E0FF74012C
:10502B006FF0E0FF75F002A42412F58274FC35F0EA
:10503B00F583E4F0A3F090FC16F090FC17F080479A
:10504B0090FC467412F0A291B3920390FC8EE0FF99
:10505B00A203E4335207EF24FF929190F811E0750D
:10506B00F002A42412F58274FC35F0F583E4F0A36E
:10507B00F0A291B3920390FC8EE0FFA203E433FE07
:10508B005207EF24FF9291C291AFE974CF5FF5E91C
:10509B00E5E930E63B90FC467410F0A291B3920325
:1050AB0090FC8EE0FFA203E4335207EF24FF9291B2
:1050BB00124668A291B3920390FC8EE0FFA203E428
:1050CB0033FE5207EF24FF9291AFE974BF5FF5E90E
:1050DB00E5E930E73B90FC467411F0A291B39203E3
:1050EB0090FC8EE0FFA203E4335207EF24FF929172
:1050FB00124668A291B3920390FC8EE0FFA203E4E8
:10510B0033FE5207EF24FF9291AFE9747F5FF5E90D
:10511B00D0D0D000D001D002D003D004D005D0061F
:10512B00D007D083D082D0F0D0E0D02132AF83E54E
:10513B008290FC43F0EFA3F090FC41E0FEA3E0FF74
:10514B0090FC43E0FCA3E0FD90FC3FE0FAA3E0FB06
:10515B008A008B011ABAFF011BE8496024EE2AF87A
:10516B00EF3BF9E82CF8E93DF9EA2CF582EB3DF53C
:10517B0083C006C007E088828983F0D007D0068001
:02518B00CF2231
:105C940000000000000001000000000000000000FF
:075CA40000000000000000F9
:10518D00AE82AF831EBEFF011FC3E49E74808FF0FD
:10519D0063F08095F050167C4C7D04EC24FFFAED05
:1051AD0034FFFB8A048B05EA4B70F080D722AE8268
:1051BD00E583CE25E0CE33FF1EBEFF011FC3E49E67
:1051CD0074808FF063F08095F040ED22AE82AF8356
:1051DD00D2919003E8C007C00612518DC291900183
:1051ED00F412518DD006D0071512AD12ED20E754F3
:1051FD00EE30E024900019C007C006C00512518D95
:10520D00D29190022612518DC29190001912518D9A
:10521D00D005D006D0078022900113C007C006C06C
:10522D000512518DD29190003212518DC291900183
:10523D001312518DD005D006D007EFC313CE13CE68
:10524D00FF1D80A8C2919003E802518DAFF0AE838F
:10525D00E58290FC4EF0EEA3F0EFA3F090FC4EE053
:10526D00FDA3E0FEA3E0FF90FC4BE0FAA3E0FBA35F
:10527D00E0FCA813A914E8496050C000C0018D825C
:10528D008E838FF01259A1F98A828B838CF012597B
:10529D00A1F8E9C398F98915D001D0006010E51582
:1052AD00F5163395E0F517851682851783220DBD0A
:1052BD0000010E90FC4EEDF0EEA3F0EFA3F00ABA54
:1052CD0000010B18B8FF011980AC90000022AFBE91
:1052DD0074FB5FF5BEE5BE30E6FBAFC674B85FF597
:1052ED00C6E5C620E6FB43BE04E5BE30E6FB53C66D
:1052FD00C743E40C43E401D2B92243FE03C2912219
:10530D00C0E0C082C083C0D090FC47E02401F0A370
:10531D00E03400F0A3E03400F0A3E03400F0D0D08E
:07532D00D083D082D0E032F2
:015CAB0001F7
:105334001245B5AF8290FC55EFF08FF005F0740183
:10534400800225E0D5F0FB90FC56F0EF75F008A440
:1053540024F9FE74F735F0FF90FC51EEF0EFA3F062
:105364008E828F83A3A374DFF08E828F83A3A3A383
:1053740074B1F08E828F83A3A3A3A3A37410F074DB
:10538400062EF582E43FF583E054E0441DF07407F3
:105394002EF582E43FF583E0543F4440F074072E39
:1053A400F582E43FF583E054FC4401F01245B5AFC7
:1053B4008290FC57EFF08FF005F07401800225E035
:1053C400D5F0FB90FC58F0EF75F008A424F9FE74B6
:1053D400F735F0FF90FC53EEF0EFA3F08E828F834D
:1053E40074DFF08E828F83A374B2F08E828F83A3D6
:1053F400A3A3A3A37410F074062EF582E43FF583EF
:10540400E054E0441EF074072EF582E43FF583E097
:1054140054CF4410F074072EF582E43FF583E05432
:10542400FC4401F043A91043B91022AF83E58290F4
:10543400FC5BF0EFA3F0E5B330E3FB90FC51E0FE3E
:10544400A3E0FF90FC5BE0FCA3E0FD8C028D038BEA
:10545400028E828F83EAF090FC51E0FEA3E0FF8E7F
:10546400828F83A37D00ECF090FC56E042D690FC42
:1054740059E0FF90FC5AE0FE4F4401F5B3E5B33028
:10548400E3FB22AF83E58290FC5FF0EFA3F090FC96
:105494005FE0FEA3E0FF90FC5DE0FCA3E0FDEC54C4
:1054A4000F60158C028D030CBC00010DEA2EF582F1
:1054B400EB3FF583E4F080E68C828D8322AF83E5B5
:1054C4008290FC66F0EFA3F090FC66E0FEA3E0FFA0
:1054D40090FC61E0FCA3E0FD90FC63E0FAA3E0FB38
:1054E40090FC65E0F990FC6FECF0EDA3F090FC719A
:1054F400EAF0EBA3F090FC73E4F090FC74E9F08E16
:10550400828F83025554AF83E58290FC6DF0EFA344
:10551400F090FC6DE0FEA3E0FF90FC68E0FCA3E0EB
:10552400FD90FC6AE0FAA3E0FB90FC6CE0F990FCCF
:105534006FECF0EDA3F090FC71EAF0EBA3F090FCBB
:10554400737402F090FC74E9F08E828F83025554D8
:10555400AF83E58290FC75F0EFA3F0E5B330E3FB95
:1055640090FC75E0FEA3E0FF90FC6FE0F519A3E06A
:10557400F51A90FC74E0FB74505BF51890FC73E032
:10558400F94B4401FB740149F51790FC71E0F513E4
:10559400A3E0F514E4F515F516C3E5159513E51622
:1055A4009514400122C00390FC51E0F8A3E0FBE510
:1055B400152EF9E5163FFA89048A058D0488828B35
:1055C40083ECF090FC51E0FCA3E0FD8C828D83A37E
:1055D400E9F090FC53E0FCA3E0FD8C828D83A3A34F
:1055E400E5152519FCE516351AFD8C028D038B0291
:1055F400EAF090FC53E0FAA3E0FB8A828B83A3A336
:10560400A3ECF090FC58E0FD90FC56E0FC4D42D633
:10561400D003E5186017E51324F0FCE51434FFFD0E
:10562400ECB51509EDB516058517B380028BB3E506
:10563400B330E3FB74102515F515E43516F51602A1
:10564400559D1256E9BC00030258B0EF60FA30D5FC
:1056540002B2D1E583B4FF030258C6E582B4FF0366
:105664000258C6258340072482400B0258B0248385
:105674001450030258C6F582EA8DF0A4A8F0EA8E0D
:10568400F0A428F8E435F0F9EB8DF0A428E935F01E
:10569400F9E433CA8FF0A429F9EA35F0FAEBF88E6D
:1056A400F0A429F9EA35F0FAE433FBEC8DF0A429EF
:1056B400F9EA35F0FAE43BFBE88FF0A42AFAEB357B
:1056C400F0FBE433CCFD8EF0A42AFAEB35F0FBE4D6
:1056D4003CFCED8FF0A42BFBEC35F0FC20E703122F
:1056E400571702588FAA82AB83A2F73392D1F5825F
:1056F4006002D2F7ACF0E58124F9F8E6FD08E6FE95
:105704000886F008E6A2F73392D5F5836002D2F753
:03571400AFF022D1
:0614BA00E478FFF6D8FD06
:105717007804EC7011E58224F8500AF582E4C9CACE
:10572700CBFCD8EF22EC7820058220E713D5820145
:1057370022C3E933F9EA33FAEB33FBEC33FCD8EA5B
:10574700158222AC82AD83AE14AF15BE0004EF60A4
:105757000C1F0FE51312580AA3DEFADFF88C828DAF
:105767008322AD82AE83AFF08D188E198F1A851301
:105777001B85141C85151DA816A9178803890418ED
:10578700B8FF0119EB4C6025851B82851C83851D9D
:10579700F01259A1FCA385821B85831C8D828E8301
:1057A7008FF0EC12580AA3AD82AE8380CE851882A3
:0757B700851983851AF02219
:101498007918E94400601B7A01905C947877759319
:1014A800FCE493F2A308B800020593D9F4DAF275C4
:0214B80093FFA0
:1057BE00FCABF0AA83A982749EC2D1F58212571750
:1057CE0002588F7F9E1257F830D1030258B0C3EFA4
:1057DE009582500974FFF5F0F583F5822279001257
:1057EE0059BD89828A838BF0EC22AA82AB83A2F701
:1057FE003392D1F5826002D2F7ACF02220F711304D
:10580E00F6138883A88220F509F6A88375830022F3
:10581E0080FEF280F5F022E5828513F0A4C582C0E9
:10582E00F08514F0A4D0F025F0C5838513F0A425DF
:10583E0083F58322E513451460467A01E51325E0CE
:10584E00F513E514334012F514E5829513E58395AF
:10585E001440030A80E6C3E51413F514E51313F59B
:10586E0013C3E5829513F5F0E58395144005F58392
:10587E0085F082C3E51413F514E51313F513DAE17D
:01588E0022F7
:1014C0007800E84400600A79007593F0E4F309D8E5
:1014D000FC7877E8440C600C790D90F000E4F0A300
:0414E000D8FCD9FA61
:02148900E4730A
:10588F00B98003EA13B34010EA2401FAE43BFBE4C6
:10589F003CFC50047C800582BC000EBB000BBA00A0
:1058AF0008E4F5F0F583F58222A2D1E582138CF09E
:1058BF0092F78B838A8222E4F583F58275F080F468
:1058CF00A2D11322E4F583F58275F0C0747F221202
:1058DF0056E930D502B2D1BF0009BC00030258D33C
:1058EF000258C6BC00030258B0E583B4FF0BE58233
:1058FF00B4FF030258D30258B0E582B4FF03025835
:10590F00C6C395835007247F400B0258B0248014E0
:10591F0050030258C6F582C3ED9AEE9BEF9C4011DF
:10592F001582C3EA33F9EB33FAEC33FBE433FC8033
:10593F0005E4CCCBCAF9C08275F019C3E99DEA9E84
:10594F00EB9FEC9400D5F002802D400EE99DF9EA13
:10595F009EFAEB9FFBEC9400FCC3B3E833F8E582AF
:10596F0033F582E58333F583C3E933F9EA33FAEB91
:10597F0033FBEC33FC80C4B3E4F938FAE43582FB33
:10598F00E43583FCD082500405827C8012571702C5
:02599F0058A707
:0D148B00758157125A00E582600302148635
:1059A10020F71430F6148883A88220F507E6A8832F
:1059B10075830022E280F7E49322E0226040F8251B
:1059C10082500274FFF582E824F8501ECCCBCAF94C
:1059D100E4CC24F85014CBCAF9E4CB24F8500BCA18
:1059E100F9E4CA24F8500379002224086010F8C3AE
:1059F100EC13FCEB13FBEA13FAE913F9D8F1227566
:035A0100820022FE
:00000001FF
